:10000000830100308A000428203084004630182004
:1000100083010730EA00E030E900463084006630B2
:100020001C2083010A128A15012804068001840A13
:100030000406031900341528F0000A128A112A2038
:100040000A128A118000840A040870060319003419
:100050001D28E900EA1B35286A1B3D286A088A002A
:100060006908E90A0319EA0A820083136A188317E8
:100070006908E90A840000080800831203136A0C67
:100080001F3903178F000313690C03178D008316A4
:100090008C170C140000000083120C08031369185D
:1000A0005828031703108C1B03140E0D831203131F
:1000B0007F39080061226D39F439E430693AF53C42
:1000C000A03673225200F43A65346639F237693249
:1000D000ED3A52100033B31233170033E412E41236
:1000E000E4125000D222D934C427CB344310D42296
:1000F000452B0026F420ED374E10A0374124412A2D
:10010000492641004F2AA0264F27301F4F104D2669
:10011000CC208024D420CD274E10CD2AD220D3202D
:10012000BD243F104400F3347238F337F934ED3A0C
:100130002810792280147529653A7937ED3A28100C
:10014000752980146C28F43AEE37F53CA03650142B
:10015000A93A4C00F43AF332F53CA0364C14A93AD3
:100160004500723BF037F53CA0364514A93A4200F1
:10017000EB30F2342810F5218014EC20693A203756
:100180004114A93A5500753774376939F53CA036E2
:100190005514F43A80146C28F430EE342810742886
:1001A0008014E526F43465376939F53CA0364D14E2
:1001B000293A4100F439F430EE342810F420801448
:1001C000F327E936F53CA0364F14A9394800F3303F
:1001D000E939F53CA0364814A9394100EE3CF43920
:1001E000F9307937ED3A2810F3228014E529793D6A
:1001F000ED3A2810F3218014F220E5396937A03553
:100200004114A9395A00F234EF357937ED3A281004
:10021000722D8014F4296F397337F934ED3A2810B0
:10022000F22980147228F330EF326932A03650146C
:1002300029394C00F63065397337F934ED3A281016
:1002400072268014F225F0346F3A20374B14293986
:10025000690069397932ED3A2810F224801472234A
:10026000EE30E939F53CA0364614293945006239AB
:10027000F934ED3A2810F2228014F225ED372810D7
:10028000F22180147221ED37281072218014F2209F
:10029000EF332037411429394E00F032753A79375F
:1002A000ED3A2810702780146F286F367937ED3AB1
:1002B00028106F2880146F2765317936ED3A2810A1
:1002C0006F278014EF2669366431EE322810EF264E
:1002D00080146F246D36F934ED3A28106F248014A1
:1002E000EF25613174362810EF218014E9216B3736
:1002F000A0375A1429374B00EC30F9302810EE297A
:10030000801461296F322037521429374D00EE30A6
:10031000E1336537203D4D14293769006437F934DE
:10032000ED3A2810EE248014752A7936ED3A28101B
:100330006D2A8014E129E1367939ED3A2810ED294A
:1003400080147228ED37F432F53CA0365014A936EB
:100350004600F232E936F53CA0364614A9364B0089
:10036000F23AF934ED3A2810ED218014ED20F23202
:10037000EB34F53CA0364114A9365400EC30F53C82
:10038000A036541429364B006F36203943142936D1
:1003900041007536E9367937ED3A2810EC208014A3
:1003A00065216B39EC32F53CA0364214A935540076
:1003B000F434EE30F53CA0365414A9345300EC3438
:1003C000F334F53CA0365314A9344E00EB34EC3230
:1003D0002810692780146926793AED3A2810692691
:1003E000801469216D3DF43A2810692180146F2A28
:1003F0007939ED3A2810682A80146F297932ED3A5C
:100400002810682980146F217234F934ED3A2810CD
:1004100068218014E529E230F237E933F53CA03653
:100420005314A9335200EE37673AEE32F53CA0364A
:100430005214A9334D00E7306537793DED3A281065
:10044000E7268014E921613B281067248014F523F6
:10045000F536A0394114A9334800E6306937F53C38
:10046000A036481429334B00EC30E634F2376937B4
:10047000F53CA036431429334B00E5396F3720375C
:100480005814A9325400EC32753620395414A9326C
:100490005300EC32EE32F53CA0365314A932520030
:1004A000EE32F53CA0365214A9324E00EF3220371E
:1004B0004E14A9324800EC32F53CA0364814A9325B
:1004C0004700F232E1367937ED3A2810E5238014FF
:1004D0006522E93620394614A9325300F232F53C40
:1004E000A0364314A9324200F232EC34F53CA03677
:1004F0004214A9325000EC3061367932ED3A2810BE
:10050000642880146527E437ED34281064278014AC
:10051000E5266437EC32F632F53CA0364D1429322C
:100520004700E430EC37EE34F53CA036471429326E
:100530004B00E430E936F53CA03643142932540030
:10054000EB326537F939ED3A2810632A8014EB292C
:10055000EE306932F53CA0365314A9314100F43530
:10056000EE34F53CA0364114A93155007537623799
:10057000F934ED3A2810F52A29316900653A6239D3
:10058000F934ED3A2810E22C8014652A6239F934E6
:10059000ED3A2810622A8014EE20693AEF362037AF
:1005A000531429315200E23AE434F53CA036521497
:1005B00029314B00F23AF5392037501429314E00D9
:1005C000F934E237F53CA0364E1429314400E23AC2
:1005D0006937F53CA036441429315400EE30613AB5
:1005E00020365414A9305200E430F53CA0365214A1
:1005F000A93050006F39613AF435EE34F53CA83635
:1006000061288014EF297932ED3A2810612780148F
:1006100061267437EE30281061268014E123793684
:10062000ED3A2810E1238014E1257336F934ED3AD0
:100630002810E121801461217939ED3A28106121D7
:100640008014F4346939F53CA03659148014752AA5
:100650006737F439EE322810A92B5600EE30E4301B
:10066000F53CA03656148014F22AEE30F53CA03644
:1006700055148014F525F53574392810A92946003C
:10068000F3376F33203950148014EB27E93965357F
:1006900020374F148014FA20F437281029275000EF
:1006A000F437F330F53CA0364B148014F934F437AA
:1006B0002810A9244800E4346F39653520374814E0
:1006C00080146C23F237281029234B00F2306F314D
:1006D0002037431480146F212039421480142010D5
:1006E00045104526D4254F296927A0252010000054
:1008A200031383120800F000003071187007031060
:1008B200F00D0310F10CF10803190800562C8312F5
:1008C2000313A4000515240E0F39F0000608F039B1
:1008D200700486008515851124080F39F00006087A
:1008E200F03970048600851585110D30A500A50B21
:1008F200782C080040300A128A112B25E030AC0017
:100902004030AD002008A900AA012930AB004930CF
:100912000A168A116F244630AB008030AC000A12EE
:100922008A110F2546300A128A112B25D630AC00C7
:100932004030AD002508A8002608A9002708AA0013
:100942002830AB0050300A168A116F240A128A111D
:100952004D30AB008030AC000A128A110F2D0A1202
:100962008A11082500300A128A112B251430AB0097
:100972004130AC000A128A110F250A30F100230817
:100982000A128A1154242207F0000A30F10070087A
:100992000A128A1154242107A00046300A128A1131
:1009A2002B25DC30AC004030AD002108A900AA01A3
:1009B2002208A700A8012308A500A6012530AB0044
:1009C20055300A168A116F240A128A115530AB006B
:1009D2008030AC000A128A110F2D83120313AD006E
:1009E2002D0E0F39F0000608F039700486008515C7
:1009F20085112D080F39F0000608F03970048600C1
:100A0200851585110D30AE00AE0B052D0800831241
:100A1200031305110130EE240230312D831203132A
:100A220005151F2D2C08EA002B08AB0A0319AC0A86
:100A32000A128A1129200A128A11EE242C08EA00CD
:100A42002B080A128A1129200A128A110038031966
:100A52000800132D83120313AB000511803EEE2C08
:100A620083120313AB000430AC005330AD00AD0B66
:100A7200382DAC0B362DAB0B342D0800831203132B
:100A820005110F303125033086008515851105309B
:100A92003125851585112130A500A50B4E2D851513
:100AA20085110530312502308600851585110D30FE
:100AB200A500A50B5A2D2830EE240830EE240F3065
:100AC200EE240630EE2CFA30312D8408031900345E
:100AD200720880008403710880008403700880001B
:100AE2000034F31F772D7814BB27782DF8018E3050
:100AF200F6008401F3080319802E0310F30CF20CA4
:100B0200F10CF00CF60A7B2D76087702031C942D6B
:100B1200031908000310F20CF10CF00CF60A760827
:100B22007702892D0310F50CF40CF30CF70A760802
:100B3200770603190800932D8030F50684015626A6
:100B4200652685257818BB27F81CAF2DF309F40913
:100B5200F509F30A0319F40A0319F50A7308F007F1
:100B620074080318740FF10775080318750FF2075C
:100B7200F801F21F802EBB277814802E8030F506F4
:100B82000008F000840A0008F100840A0008F2005C
:100B9200A02D7208750680390319D32D750D7508BD
:100BA20001380800F21375087F397202031DE12D26
:100BB20074087102031DE12D730870020319080005
:100BC20003080238F51B013A830003188038080035
:100BD200840156266526F901FA01FB010730F5006A
:100BE2000310F40CF30C031C012E7008F9077108B2
:0E0BF2000318710FFA0772080318720FFB0741
:100C00000310F00DF10DF20DF50BF12D0930F5008B
:100C10000D2E0310FB0CFA0CF90C0310F40CF30C62
:100C2000031C1C2E7008F90771080318710FFA07CE
:100C300072080318720FFB07F50B092E7A3077073D
:100C4000F607780CF8067908F0007A08F1007B08BE
:100C5000F200802E0008F000840A0008F100840AE7
:100C60000008F200EA2D84015626F3018230F607CF
:100C7000F61B612EF030F607F61B4F2E1830760269
:100C80000318612EF608031D482E7818BB270800AC
:100C9000F6030310F00DF10DF20DF30D422E0310CB
:100CA000F20CF10CF00CF60F4F2E452EF801710DE1
:100CB000720DF60000380319612EF80DF201F117DC
:100CC0000800F001F101F2010034F810740D750D07
:100CD000F70000380319712E0318F814F501F41702
:100CE0000800F701F301F401F50108007608031983
:100CF000612EF113F80C760CF2000318F117662D33
:100D0000F608031D942EF001F101F201662D720325
:100D10000319F00A0319F10A0319F20A0310F20C7D
:100D2000F10CF00CF60A802EF208031D872E7008D5
:100D300071040319832EF11B762EF6030310F00DB8
:100D4000F10D9B2E0008F000840A0008F100840ACF
:100D50000008F200840A0008F300AF2E8401831219
:100D60000313E601F801F901FA01FB0174087504A7
:100D7000760477040319BF2EC030E605CA2EF001B1
:100D8000F101F201F301C92F0310F40DF50DF60D79
:100D9000F70DE60AF71FC42EE60A0310F80DF90D49
:100DA000FA0DFB0D77087302031DE02E7608720220
:100DB000031DE02E75087102031DE02E74087002F9
:100DC000031CF22E78147408F0027508031C750FCA
:100DD000F1027608031C760FF2027708031C770FE6
:100DE000F3020310F70CF60CF50CF40CE60366089E
:100DF0003F39031DCD2E661F0A2F0310FF30F00769
:100E0000F009031CF107F109031CF207F209031CA6
:100E1000F307F3097008F4007108F5007208F60092
:100E20007308F7007808F0007908F1007A08F200FA
:100E30007B08F300E61FC92F0310FF30F007F0090D
:100E4000031CF107F109031CF207F209031CF30765
:100E5000F309C92F84017008F8007108F9007208BD
:100E6000FA007308FB00F201F301F001F101031035
:100E7000FB0CFA0CF90CF80C031C4C2F7408F0074F
:100E800075080318750FF10776080318760FF20737
:100E900077080318770FF307780879047A047B043E
:100EA0000319C92F0310F40DF50DF60DF70D372FAB
:100EB0000008F000840A0008F100840A0008F2002B
:100EC000840A0008F3002B2F83120313E801720D2C
:100ED000730DE60000380319712FE80DF301F217C6
:100EE0000800F001F101F201F3010034E810760D81
:100EF000770DE70000380319822F0318E814F70173
:100F0000F6170800E701F401F501F601F701080002
:100F100066080319712FF213E80C660CF30003182E
:100F2000F217C92FE6080319B62F73080319A82F63
:100F300073030319F00A0319F10A0319F20A0319DA
:100F4000F30A0310F30CF20CF10CF00CE60A922FEA
:100F500070087104720473040319B62FF21B882FF2
:100F6000E6030310F00DF10DF20DAE2FF001F101CB
:100F7000F201F301C92F0310FF30F007F009031C41
:100F8000F107F109031CF207F209031CF307F30947
:100F90000800840803190034730880008403720871
:100FA000800084037108800084037008800000348E
:100FB000710D720D0038031908008030F206080028
:100FC00041344E343A3420342034203400344B340D
:100FD0004E343A3420342034203420340034203449
:100FE0002034203420342034203420342034203461
:100FF0002034203420342034203420342034003471
:1010020083160313860185010F30870006309F0087
:101012008312850186018701FA300A128A1131256D
:101022000A128A113F250A128A1108250C300A1267
:101032008A11EE2400300A128A112B25DE30AB0011
:101042004630AC000A128A110F2540300A128A116A
:101052002B25E330AB004030AC000A128A110F2579
:10106200A4010A128A1164250A128A15A40A0830F8
:101072002402031C32280A128A11082500300A129F
:101082008A112B251430AB004130AC000A128A11B0
:101092000F250A128A15A301A201A101071C5E28CD
:1010A200A30A0A128A1164252308023A0319A3012A
:1010B2000A128A11B0240A128A15871C6D28A20A04
:1010C2000A128A11642522080A3A0319A2010A1295
:1010D2008A11B0240A128A15071D7C28A10A0A1255
:1010E2008A11642521080A3A0319A1010A128A11F8
:1010F200B0240A128A15871D4F280A128A11082560
:1011020000300A128A112B250A128A15A008031D23
:101112008E280330AB004130F52F200B9F28B530CD
:10112200AB004630AC000A128A110F250A128A154A
:10113200E530A5008030A6003F30AF282008023AF3
:10114200031DB628B530AB004430AC000A128A1138
:101152000F251030A5008030A6004030A7000A12EB
:101162008A117B240A128A15F92F2008033A031DDB
:10117200C728D630AB004330AC000A128A110F25C3
:101182000A128A151D30A500DE30AD282008043A67
:10119200031DD828E730AB004430AC000A128A1194
:1011A2000F250A128A153130A50010309229200825
:1011B200053A031DE928D630AB004630AC000A12CE
:1011C2008A110F250A128A15FA30A5002C309229AD
:1011D2002008063A031DFA28CB30AB004630AC009B
:1011E2000A128A110F250A128A152D30A5004030E5
:1011F20092292008073A031D0B299630AB0046308E
:10120200AC000A128A110F250A128A151930A5009C
:10121200603092292008083A031D1C298A30AB004D
:101222004630AC000A128A110F250A128A15FC30C8
:10123200A5007F3092292008093A031D2D29C230CA
:10124200AB004630AC000A128A110F250A128A1529
:10125200FC30A5009730922920080A3A031D3E2946
:10126200AB30AB004430AC000A128A110F250A12CF
:101272008A156F30A500A130922920080B3A031D70
:101282004F290430AB004630AC000A128A110F25F8
:101292000A128A15E930A500B730922920080C3AC3
:1012A200031D60293530AB004430AC000A128A11AC
:1012B2000F250A128A157130A500C2309229200822
:1012C2000D3A031D71299130AB004330AC000A1274
:1012D2008A110F250A128A15D930A500D730922912
:1012E20020080E3A031D8229BD30AB004330AC000A
:1012F2000A128A110F250A128A15AE30A500E030B3
:10130200922920080F3A031D95297F30AB00463001
:10131200AC000A128A110F250A128A15C930A500DB
:10132200F730A6004130AF282008103A031DA62945
:101332007430AB004630AC000A128A110F250A1233
:101342008A153D30A500A601B7292008113A031DD0
:10135200B9298730AB004330AC000A128A110F253D
:101362000A128A15CF30A5000D30A6004230AF28F0
:101372002008123A031DCA298E30AB004230AC005D
:101382000A128A110F250A128A15CB30A5001F30C6
:10139200B6292008133A031DDB299F30AB004630E3
:1013A200AC000A128A110F250A128A156430A500B0
:1013B2001C30B6292008143A031DEC292830AB0052
:1013C2004630AC000A128A110F250A128A155030D3
:1013D200A5002030B6292008153A031DFD294E30FC
:1013E200AB004530AC000A128A110F250A128A1589
:0E13F200D230A5003330B6292008163A031D6C
:101400000E2AAF30AB004330AC000A128A110F2510
:101410000A128A158530A5003F30B6292008173AF0
:10142000031D1F2A5B30AB004630AC000A128A1144
:101430000F250A128A15C430A5004B30B6292008A2
:10144000183A031D302A7A30AB004230AC000A1241
:101450008A110F250A128A15FC30A5004F30B629D3
:101460002008193A031D412A0D30AB004330AC006F
:101470000A128A110F250A128A15C130A5005B30A5
:10148000B62920081A3A031D522AD030AB00443046
:10149000AC000A128A110F250A128A156330A500C2
:1014A0005F30B62920081B3A031D632AE030AB00E9
:1014B0004230AC000A128A110F250A128A15BB307D
:1014C000A5006B30B62920081C3A031D742ACB30C6
:1014D000AB004330AC000A128A110F250A128A159C
:1014E000C830A5006A30B62920081D3A031D852A98
:1014F0006F30AB004130AC000A128A110F250A127E
:101500008A152F30A5007E30B62920081E3A031D0B
:10151000962AEC30AB004230AC000A128A110F253B
:101520000A128A15C830A5008230B62920081F3A51
:10153000031DA72A1C30AB004630AC000A128A11EA
:101540000F250A128A157230A5008B30B6292008A3
:10155000203A031DB82AC130AB004430AC000A1257
:101560008A110F250A128A153830A5009130B62944
:101570002008213A031DC92AF830AB004130AC00E5
:101580000A128A110F250A128A15D830A500953043
:10159000B6292008223A031DDA2A9130AB004430E4
:1015A000AC000A128A110F250A128A15EC30A50028
:1015B0009D30B6292008233A031DEB2A8430AB0066
:1015C0004230AC000A128A110F250A128A15CF3058
:1015D000A5009F30B6292008243A031DFC2A443078
:1015E000AB004230AC000A128A110F250A128A158C
:1015F0009A30A500A730B6292008253A031D0D2BE7
:10160000A530AB004530AC000A128A110F250A1232
:101610008A15EF30A500AA30B6292008263A031D06
:101620001E2B1430AB004230AC000A128A110F2579
:101630000A128A153D30A500AF30B6292008273A96
:10164000031D2F2B4230AB004630AC000A128A112A
:101650000F250A128A15CF30A500B130B62920080F
:10166000283A031D402B0530AB004230AC000A1273
:101670008A110F250A128A157330A500B630B629D3
:101680002008293A031D512BBF30AB004530AC0078
:101690000A128A110F250A128A15D030A500B93016
:1016A000B62920082A3A031D622BC430AB00423011
:1016B000AC000A128A110F250A128A15E130A50022
:1016C000BF30B62920082B3A031D722B3F30AB00E8
:1016D0004530AC000A128A110F250A128A15A5019D
:1016E000C430B62920082C3A031D832B3630AB00BA
:1016F0004130AC000A128A110F250A128A152430D3
:10170000A500CA30B62920082D3A031D942BFA30C3
:10171000AB004330AC000A128A110F250A128A1559
:10172000CF30A500CD30B62920082E3A031DA52BB9
:10173000F530AB004430AC000A128A110F250A12B2
:101740008A15D730A500D430B62920082F3A031DBA
:10175000B62B4E30AB004430AC000A128A110F2574
:101760000A128A15BC30A500D730B6292008303AB5
:10177000031DC72B3130AB004530AC000A128A1173
:101780000F250A128A15D230A500E030B6292008AC
:10179000313A031DD82B1B30AB004330AC000A128A
:1017A0008A110F250A128A15A430A500E530B62942
:1017B0002008323A031DE92BF730AB004230AC0071
:1017C0000A128A110F250A128A156C30A500ED3015
:1017D000B6292008333A031DFA2B9830AB00453068
:1017E000AC000A128A110F250A128A158430A5004E
:1017F000F330B6292008343A031D0B2C8530AB009A
:101800004430AC000A128A110F250A128A153330AF
:10181000A500FF30B6292008353A031D1C2CAC303A
:10182000AB004630AC000A128A110F250A128A1545
:10183000CF30A500FD30B6292008363A031D2D2CE7
:101840007930AB004430AC000A128A110F250A121D
:101850008A154A30A5000330702C2008373A031D42
:101860003E2CEC30AB004130AC000A128A110F253F
:101870000A128A15E830A5000430702C2008383A86
:10188000031D4F2C3630AB004630AC000A128A11D3
:101890000F250A128A155430A5000930702C200833
:1018A000393A031D602C1030AB004630AC000A12F0
:1018B0008A110F250A128A15E830A5000A30702C0B
:1018C00020083A3A031D732CDB30AB004430AC00E7
:1018D0000A128A110F250A128A151D30A5000C3034
:1018E000A6004330AF2820083B3A031D822C243049
:1018F000AB004230AC000A128A110F250A128A1579
:10190000E8306E2C20083C3A031D932C0430AB00C9
:101910004530AC000A128A110F250A128A153D3093
:10192000A5001030702C20083D3A031DA32C423036
:10193000AB004330AC000A128A110F250A128A1537
:10194000A5011130702C20083E3A031DB42C343010
:10195000AB004330AC000A128A110F250A128A1517
:101960005C30A5001630702C20083F3A031DC52CB2
:101970006130AB004130AC000A128A110F250A1207
:101980008A15F730A5001730702C2008403A031D47
:10199000D62C2130AB004530AC000A128A110F253D
:1019A0000A128A154030A5001D30702C2008413ADB
:1019B000031DE72C8A30AB004530AC000A128A11B7
:1019C0000F250A128A15ED30A5001E30702C200854
:1019D000423A031DF82C2530AB004130AC000A120E
:1019E0008A110F250A128A158030A5002230702C2A
:1019F0002008433A031D092DD230AB004230AC0021
:101A00000A128A110F250A128A15EE30A500243019
:101A1000702C2008443A031D1A2D6D30AB00423063
:101A2000AC000A128A110F250A128A154330A5004C
:101A30002730702C2008453A031D2B2D2830AB0091
:101A40004330AC000A128A110F250A128A15EF30B2
:101A5000A5002830702C2008463A031D3C2D7B3011
:101A6000AB004530AC000A128A110F250A128A1504
:101A70000A30A5002D30702C2008473A031D4D2D4B
:101A80005330AB004130AC000A128A110F250A1204
:101A90008A15F830A5002E30702C2008483A031D16
:101AA0005E2D5930AB004430AC000A128A110F256C
:101AB0000A128A157D30A5003230702C2008493A70
:101AC000031D6F2DDB30AB004530AC000A128A11CC
:101AD0000F250A128A15F230A5003430702C200828
:101AE0004A3A031D802D4E30AB004630AC000A123E
:101AF0008A110F250A128A15DA30A5003730702CAA
:101B000020084B3A031D912D9F30AB004430AC00B0
:101B10000A128A110F250A128A153530A5003A30AB
:101B2000702C20084C3A031DA22DC030AB00413070
:101B3000AC000A128A110F250A128A153330A5004B
:101B40003E30702C20084D3A031DB32D5130AB00B0
:101B50004230AC000A128A110F250A128A15383059
:101B6000A5004030702C20084E3A031DC52D96303C
:101B7000AB004130AC000A128A110F250A128A15F7
:101B80001430A5004330A600AF2820084F3A031DAB
:101B9000D62D7A30AB004130AC000A128A110F25E5
:101BA0000A128A15F730A5004430702C2008503AEC
:101BB000031DE72D4430AB004430AC000A128A11FB
:101BC0000F250A128A159730A5004830702C20087E
:101BD000513A031DF82D7B30AB004330AC000A12A4
:101BE0008A110F250A128A156230A5004C30702C1C
:101BF0002008523A031D092EB330AB004530AC002B
:101C00000A128A110F250A128A153330A5004F30A7
:101C1000702C2008533A031D1A2EE230AB004330DB
:101C2000AC000A128A110F250A128A15FB30A50092
:101C30005030702C2008543A031D2A2EA830AB00D7
:101C40004230AC000A128A110F250A128A15A5012A
:101C50005130702C2008553A031D3A2EB330AB009A
:101C60004130AC000A128A110F250A128A15A5010B
:101C70005230702C2008563A031D4A2E0230AB0019
:101C80004330AC000A128A110F250A128A15A501E9
:101C90005E30702C2008573A031D5A2E5E30AB0080
:101CA0004230AC000A128A110F250A128A15A501CA
:101CB0005F30702C2008583A031D6B2EE730AB00C4
:101CC0004530AC000A128A110F250A128A15063017
:101CD000A5006230702C2008593A031D7B2E5D3020
:101CE000AB004530AC000A128A110F250A128A1582
:101CF000A5016330702C20085A3A031D8C2EEE305B
:101D0000AB004330AC000A128A110F250A128A1563
:101D10000A30A5006830702C20085B3A031D9D2E08
:101D2000F330AB004530AC000A128A110F250A12BD
:101D30008A150930A5006730702C20085C3A031D15
:101D4000AE2E6830AB004630AC000A128A110F2567
:101D50000A128A150730A5006E30702C20085D3AF3
:101D6000031DBF2E9930AB004230AC000A128A111D
:101D70000F250A128A150C30A5006D30702C200832
:101D80005E3A031DCF2E4430AB004130AC000A1246
:101D90008A110F250A128A15A5017430702C2008AB
:101DA0005F3A031DDF2E6C30AB004330AC000A12EB
:101DB0008A110F250A128A15A5017330702C20088C
:101DC000603A031DE72E5F30AB004330EE2E200853
:101DD000613A031DF72EA030AB004330AC000A126D
:101DE0008A110F250A128A15A5017730702C200858
:101DF000623A031D072F6730AB004430AC000A1273
:101E00008A110F250A128A15A5017B30702C200833
:101E1000633A031D172FDB30AB004130AC000A12D0
:101E20008A110F250A128A15A5017C30702C200812
:101E3000643A031D272F5130AB004330AC000A1227
:101E40008A110F250A128A158030A500702C2008EF
:101E5000653A031D362F1030AB004530AC000A1236
:101E60008A110F250A128A15A501452F2008663A06
:101E7000031D472FB630AB004230AC000A128A1166
:101E80000F250A128A158030A5008130702C200899
:101E9000673A031D562F3330AB004230AC000A12B4
:101EA0008A110F250A128A15A501652F2008683AA4
:101EB000031D672FC530AB004030AC000A128A11F9
:101EC0000F250A128A158030A5008230702C200858
:101ED000693A031D6F2FCD30AB004530862F2008A7
:101EE0006A3A031D7F2F1430AB004430AC000A1255
:101EF0008A110F250A128A158030A5008D2F20081F
:101F00006B3A031D8F2F0630AB004430AC000A1231
:101F10008A110F250A128A15A5018330702C20081A
:101F20006C3A031DA02FCD30AB004130AC000A123B
:101F30008A110F250A128A158030A5008430702C72
:101F400020086D3A031DB02FA230AB004130AC0029
:101F50000A128A110F250A128A15A5018530702CE4
:101F600020086E3A031DC12FB430AB004030AC00E6
:101F70000A128A110F250A128A158030A5008730AF
:101F8000702C20086F3A031DD12F2530AB00443050
:101F9000AC000A128A110F250A128A15A501883091
:101FA000702C2008703A031DE22F6B30AB004530D7
:101FB000AC000A128A110F250A128A158030A5007A
:101FC0008A30702C2008713A031DF22F8530AB0047
:101FD0004130AC000A128A110F250A128A15A50198
:101FE0008E30702CF430AB004030AC000A128A11F5
:101FF0000F25FA300A128A1131250A128A154C2847
:1028DE0083120313B500B1012B08AF00E82F3408A3
:1028EE00253A031DD92FFF30B300B201B001952F49
:1028FE00B5080319862C350884008313800131082E
:10290E0008000230AF072F02840083130008D72F70
:10291E00B017952FB00A972C0830B307FE30B307C7
:10292E00B01FA92C0430AF072F02840083130008B8
:10293E00F000840A0008F100840A0008F200840AFC
:10294E000008B92C0230AF072F0284008313000851
:10295E00F000840A0008F100700871080030F11BC5
:10296E00FF30F200F3007008BE007108BF0072085D
:10297E00C0007308C100301CE32CC11FF22C3E08AE
:10298E00F0003F08F1004008F2004108F300F009A2
:10299E00F109F209F309F00A0319F10A0319F20A0F
:1029AE000319F30A7008BE007108BF007208C00058
:1029BE007308C100B203F32CB01BF22C3F08F100D8
:1029CE003E08F000F201F301BE007108BF0072086C
:1029DE00C0007308C100B0010B30B3073308F40018
:1029EE00F501F601F7013E08F0003F08F10040083E
:1029FE00F2004108F3000A128A11AE267408B400E0
:102A0E003308F400F501F601F7013E30840083131C
:102A1E000A128A11A2260A168A1183120313C20100
:102A2E00C20AC301C401C50145084102031D292D77
:102A3E0044084002031D292D43083F02031D292D82
:102A4E0042083E02031C572D3308F400F501F6012F
:102A5E00F7014230840083130A128A1158270A168E
:102A6E008A1183120313B2031B2DB10AB508031981
:102A7E004D2D3508840083133019472D2030482DF5
:102A8E003030800083120313B50A572D3019512DA3
:102A9E002030522D30300A128A1151240A168A1112
:102AAE00B2033208803A7F3E03183C2D301C6E2D47
:102ABE00B10AB50803196A2D3508840083132D3029
:102ACE008000B50A6E2D2D300A128A11512433085A
:102ADE00F400F501F601F7014230840083130A1267
:102AEE008A11A2260A168A117308720471047004E0
:102AFE000319B52D831203134208F4004308F500A1
:102B0E004408F6004508F7003E08F0003F08F100C3
:102B1E004008F2004108F3000A128A11AE2633086B
:102B2E00F400F501F601F7010A128A11AE260A1613
:102B3E008A117408B200803A763E031CA82D073025
:102B4E00B207B10AB5080319B22D350884008313F4
:102B5E003208303E672D3208303E6B2D0A3083121C
:102B6E0003133402031CBD2D0730B407B10AB50898
:102B7E000319C92D3508840083133408303E8000B4
:102B8E00B50AD02D3408303E0A128A1151240A1685
:102B9E008A11B01CE82FB10AB5080319DD2D3508CE
:102BAE00840083132E308000B50AE32D2E300A12D6
:102BBE008A1151240A168A113608BE003708BF0042
:102BCE003808C0003908C1000430B0002E08B20029
:102BDE00DB2E0330AF072F02840083130008C200E0
:102BEE00840A0008C300840A0008C40007303302B8
:022BFE00031CB6
:102C0000032E0630B3003308AE00B001F301F40127
:102C1000F5014208F0004308F1004408F2000A12EE
:102C20008A11CA250A168A110318292EB001B00A82
:102C30004208F0004308F1004408F2000A128A1129
:102C4000D8270A168A117008C2007108C3007208DA
:102C5000C400AE08031D472E4208F3004308F400E9
:102C60004408F500F001F1013F30F2000A128A1128
:102C70009F250A128A1133260A168A117008BE008F
:102C80007108BF007208C0007308C100DB2E2E0A55
:102C9000B2024208F0004308F1004408F2000A12B0
:102CA0008A1133267008BE007108BF007208C00088
:102CB0007308C1003E08F0003F08F1004008F20030
:102CC0004108F3000A128A1177257008F300710891
:102CD000F4007208F5004230840083130A128A114E
:102CE000BF2583120313B014BA01BA0ABB01BC0199
:102CF000BD01F3012030F4004130F5004230840082
:102D000083130A128A112A260A30F400F501F6010B
:102D1000F701831203133A30840083130A128A11D5
:102D200058270A168A1183120313B30B792EF30165
:102D3000F4013F30F5004230840083130A128A11F7
:102D4000C125831203134208F0004308F100440830
:102D5000F2000A128A1133260A168A117008B60088
:102D60007108B7007208B8007308B9003D0839024D
:102D7000031DC42E3C083802031DC42E3B08370235
:102D8000031DC42E3A083602031CDB2E3A08B60295
:102D90003B08031C3B0FB7023C08031C3C0FB80266
:102DA0003D08031C3D0AB902BE0A0319BF0A0319F4
:102DB000C00A0319C10A0A30B300F52CB10AB508DC
:102DC0000319E92E35088400831320308000B50AEA
:102DD000EF2E20300A128A1151240A168A11B203EA
:102DE0003208803A7E3E0318DE2E0230AF072F02F3
:102DF000840083130008B400D92F0230AF072F02DC
:102E0000840083130008C200840A0008C300B401D0
:102E100034084207E9004308EA0069080318EA0A8F
:102E20000A128A1129200A168A11003803191A2F4A
:102E3000B40A082F330834020318202F3408B300D3
:102E40003308B21B572FFF3A3207031C572FB10A22
:102E5000B5080319322F3508840083132030800011
:102E6000B50A382F20300A128A1151240A168A1105
:102E7000B203202F4308EA0042080A128A112920CF
:102E80000A168A11B400C20A0319C30AB10AB508A6
:102E90000319512F35088400831334088000B50AC4
:102EA000572F34080A128A1151240A168A11B303C3
:102EB000330F3A2FE82F2D08EA002C080A128A1146
:102EC00029200A168A112A3A031D6D2F0230AF07F6
:102ED0002F02840083130008912F2D08EA002C088C
:102EE0000A128A112920D03EB300AC0A0319AD0A98
:102EF0002D08EA002C080A128A1129200A168A11C4
:102F0000B40030303402031C952F3A3034020318D9
:102F1000952F0A30F10033080A128A11542434071D
:102F2000D03EB300AC0A0319AD0A2D08EA002C0804
:102F3000AC0A0319AD0A0A128A1129200A168A114D
:102F4000B400003A03197F2C2A3A0319882C043A5A
:102F500003195B2F763A0319932C3B3A0319F02E91
:102F6000073A0319912C023A0319F02D0A3A031972
:102F70008F2C033A0319952C1C3A0319FD2E063A9F
:102F80000319972C0D3A0319932C30303402031C8B
:102F9000D92F3A3034020318D92F0A30F100320801
:102FA0000A128A1154240A168A113407D03EB2003C
:102FB000952FB10AB5080319E42F3508840083134F
:102FC00034088000B50AE82F34080A128A11512407
:102FD0002D08EA002C08AC0A0319AD0A0A128A115E
:102FE00029200A168A11B400B408031D762CB508EE
:102FF0000319FE2F3508840083138001310808006F
:02400E0071FF40
:00000001FF
